:020000040000FA
:0A000000000000008AEF00F0A2D01B
:08001800EFD09EA8FED7AD6EEB
:100020001200126E960E096E980E0A6E4CD8D8B455
:10003000CA90D8A4CA80FC0FD8A0CA92D8B0CA82ED
:10004000800E096E960E0A6E980E0D6E0E6ACAB07C
:100050001CD8CAB21AD839D80904CB6E09C00BF023
:100060000AC00CF002500F6E106E023C106A42D8AB
:100070000E50122E0AD0BE6E0C0EBD6E0DBEBD8A85
:100080000DBCBD889494CA84120000D8D8900D325B
:100090000A32093212000C6A0B6EFF0E0B260C227C
:1000A00000D0D8A01200030E0A6EE60E02D8F5D7D3
:1000B0000A6AFE0F096EE86A0A5AD8A01200000008
:1000C000090600D0F8D70E6A0D6A100EF36E0A34D6
:1000D0000D360E360B500D5C0C500E5805E30B50D0
:1000E0000D5E0C500E5AD88009360A36F32EEFD723
:1000F000095012000B500F02F3CF0DF0F4CF0EF0A9
:100100000C500F02F3500E260B501002F3500E2627
:100110000D501200006A4F0EAF6E240EAC6E900EA2
:10012000AB6E00010F0EC16E070EB46E0FEE7FF0C6
:10013000ED6AE950EA10FCE1EF6AC69AC30E926ECE
:10014000E00E936EC00E946E928092826AD0F2A4FA
:1001500003D0F294817A11009EAA19D0060EAB1436
:1001600012E1E2CF3DF0E1CF3CF03E2A10EE5CF030
:100170003E50E126000EE222AECFE7FF3DC0E2FF97
:100180003CC0E1FF1100AE50AE50AB98AB881100FF
:100190003E503F5C14E03F2AEACF0AF0E9CF09F075
:1001A00000EE5CF03F50E926000EEA22EF503B6E75
:1001B0000AC0EAFF09C0E9FFD880120004D0E8684D
:1001C0003B6ED8A0120012003E6A3F6A9D8A9F8A49
:1001D000F28EF28C12009D9A00EE5CF0010EF46E2D
:1001E000F36AF306000EF45AEE6AF450F310F9E1E4
:1001F0003E6A3F6A9D8A1200F29EE0CF5CF4D8CF3F
:100200005DF4E8CF5EF4F28E0001A192B36AB26AA7
:10021000F29E5CC4E0FF5DC4D8FF5EC4E8FFF28ECE
:100220001000939A8A8A0A0E36DF939A8A9A9298D5
:10023000899893948A94929A899A94908B909492A4
:100240008B9294948B9494968B9694988B98949A82
:100250008B9A276A256A00EE40F01C0EEE68E82EA5
:10026000FDD7266A7F0E2F6EAFDFB5DFCD6AF29421
:10027000F28A870ED56EB16AA192A082B36AB26A81
:10028000D08EA292B10EB16EA2EC06F09FEC0AF0F5
:10029000342AE86A34B2010F35B0010806E135703E
:1002A000302A000E31223222332272DF3BC016F098
:1002B000C00E165C07E3FE0E165C01E301D0186A5F
:1002C0005EEF04F016AE38D0186A8F0E165C05E1AA
:1002D00016C018F019681A682DD09F0E165C05E13B
:1002E00016C018F01B681C6825D0AF0E165C05E11F
:1002F00016C018F01D681E681DD0BF0E165C05E103
:1003000016C018F01F68206815D0CF0E165C04E1E7
:1003100016C018F021680ED0DF0E165C04E116C07E
:1003200018F0226807D0EF0E165C04E116C018F032
:10033000236824685DEF04F0185204E15EEF04F0D6
:100340005DEF04F08F0E185CD8A48AD0192803E161
:1003500016C019F081D016C01AF0180E195C07E10A
:100360008F0E5BDE180E59DE1A5057DE72D0190E52
:10037000195C07E18F0E51DE190E4FDE1A504DDE6B
:1003800068D01C0E195C07E18F0E47DE195045DE60
:10039000000E43DE5ED02A0E195C0AE3550E195C8E
:1003A00007E28F0E3ADE195038DE1A5036DE51D091
:1003B000600E195C08E1899A25902790436842688D
:1003C0004168406846D0610E195C08E18B90259227
:1003D000279247684668456844683BD0620E195CBE
:1003E00003E0630E195C07E18F0E17DE195015DE6E
:1003F000000E13DE2ED0780E195C0EE18B92026A8D
:10040000520E0C6E080E0B6E010E0BDE25964F6819
:100410004E684D684C681DD07A0E195C02E18B96CF
:1004200018D07B0E195C08E18B98259A279A57689B
:100430005668556854680DD07C0E195C08E18B9A9B
:10044000259C279C5B685A685968586802D05EEF03
:1004500004F019685DEF04F05EEF04F05DEF04F066
:100460009F0E185CD8A4EED11B2803E116C01BF028
:10047000E7D116C01CF01C52D8A48DD0180E1B5CFE
:100480000AE19F0E0DEC00F0180E0DEC00F0000ECE
:100490000DEC00F07ED0190E1B5C0AE19F0E0DECF6
:1004A00000F0190E0DEC00F0000E0DEC00F071D014
:1004B0001C0E1B5C0AE19F0E0DEC00F01B500DECB6
:1004C00000F0000E0DEC00F064D02A0E1B5C0DE372
:1004D000550E1B5C0AE29F0E0DEC00F01B500DEC5C
:1004E00000F0000E0DEC00F054D0600E1B5C08E133
:1004F000899A25902790436842684168406849D0AE
:10050000610E1B5C08E18B90259227924768466834
:10051000456844683ED0620E1B5C03E0630E1B5CC2
:100520000AE19F0E0DEC00F01B500DEC00F0000EE8
:100530000DEC00F02ED0780E1B5C0FE18B92026A5E
:10054000520E0C6E080E0B6E010E11EC00F025968B
:100550004F684E684D684C681CD07A0E1B5C02E1F7
:100560008B9617D07B0E1B5C08E18B98259A279AF7
:1005700057685668556854680CD07C0E1B5C08E1BF
:100580008B9A259C279C5B685A685968586801D0EB
:1005900095D193D155D126A051D1180E1B5C0AE1FB
:1005A0009F0E0DEC00F0180E0DEC00F01C500DEC41
:1005B00000F044D1190E1B5C0AE19F0E0DEC00F017
:1005C000190E0DEC00F01C500DEC00F037D11C0E94
:1005D0001B5C0AE19F0E0DEC00F01B500DEC00F0CF
:1005E0001C500DEC00F02AD12A0E1B5C0DE3550EB9
:1005F0001B5C0AE29F0E0DEC00F01B500DEC00F0AE
:100600001C500DEC00F01AD1600E1B5C2FE11CC0D9
:1006100029F0898A7F0E295C22E2278003EE5CF0B4
:10062000D8902934E926000EEA22EECF07F0EFCF6A
:1006300008F007503024036E08503120046E000E7D
:100640003220056E000E3320066E06C043F005C052
:1006500042F004C041F003C040F0258006D027904E
:1006600025904368426841684068E8D0610E1B5C91
:100670002FE11CC02AF08B807F0E2A5C22E22782A9
:1006800003EE5CF0D8902A34E926000EEA22EECF81
:1006900007F0EFCF08F007503024036E08503120E8
:1006A000046E000E3220056E000E3320066E06C06A
:1006B00047F005C046F004C045F003C044F0258271
:1006C00006D0279225924768466845684468B6D0A8
:1006D000620E1B5C03E0630E1B5C0AE19F0E0DECD7
:1006E00000F01B500DEC00F01C500DEC00F0A6D0FB
:1006F000780E1B5C38E18B822FC002F0520E0C6E1C
:10070000080E0B6E010E11EC00F01CC02BF07F0EDA
:100710002B5C22E2278602EE5CF0D8902B34E9268F
:10072000000EEA22EECF07F0EFCF08F0075030249A
:10073000036E08503120046E000E3220056E000E4C
:100740003320066E06C04FF005C04EF004C04DF0D9
:1007500003C04CF0258606D0279625964F684E6834
:100760004D684C686BD07A0E1B5C02E18B8666D0BC
:100770007B0E1B5C2FE11CC02CF08B887F0E2C5C49
:1007800022E2278A02EE5CF0D8902C34E926000E93
:10079000EA22EECF07F0EFCF08F007503024036EC7
:1007A00008503120046E000E3220056E000E3320FA
:1007B000066E06C057F005C056F004C055F003C0E1
:1007C00054F0258A06D0279A259A576856685568A6
:1007D000546834D07C0E1B5C2FE11CC02DF08B8A3A
:1007E0007F0E2D5C22E2278C02EE5CF0D8902D3437
:1007F000E926000EEA22EECF07F0EFCF08F007500F
:100800003024036E08503120046E000E3220056E35
:10081000000E3320066E06C05BF005C05AF004C01F
:1008200059F003C058F0258C06D0279C259C5B68A6
:100830005A685968586802D01B6840D01B683DD080
:100840003DD03BD0AF0E185C0BE11D2803E116C074
:100850001DF004D016C01EF081D92FD02FD02DD07E
:10086000BF0E185C0AE11F2803E116C01FF003D079
:1008700016C020F0A8D922D020D0CF0E185C07E1F6
:10088000212803E116C021F0216818D016D0DF0E10
:10089000185C07E1222803E116C022F092D90ED09D
:1008A0000CD0EF0E185C09E1232803E116C023F0F9
:1008B00003D016C024F083D901D016D9070E3A5CB4
:1008C000D8B009D13650305C375031583850325892
:1008D00039503358D8A0F1D0398E3A522AE127B096
:1008E00006D0899A436842684168406821D0807A7E
:1008F000929A03EE5CF0D8902934E926000EEA22A1
:10090000EECF07F0EFCF08F007503024036E085009
:100910003120046E000E3220056E000E3320066E6C
:1009200006C043F005C042F004C041F003C040F0EF
:10093000C3D0010E3A5C2AE127B206D08B904768FB
:1009400046684568446821D08270949003EE5CF05C
:10095000D8902A34E926000EEA22EECF07F0EFCF36
:1009600008F007503024036E08503120046E000E4A
:100970003220056E000E3320066E06C047F005C01B
:1009800046F004C045F003C044F096D0020E3A5C35
:1009900005E14B684A68496848688ED0030E3A5CA6
:1009A0002AE127B606D08B924F684E684D684C6896
:1009B00021D08272949202EE5CF0D8902B34E9261A
:1009C000000EEA22EECF07F0EFCF08F007503024F8
:1009D000036E08503120046E000E3220056E000EAA
:1009E0003320066E06C04FF005C04EF004C04DF037
:1009F00003C04CF061D0040E3A5C05E153685268C4
:100A00005168506859D0050E3A5C2AE127BA06D0E1
:100A10008B98576856685568546821D082789498A6
:100A200002EE5CF0D8902C34E926000EEA22EECFDC
:100A300007F0EFCF08F007503024036E0850312044
:100A4000046E000E3220056E000E3320066E06C0C6
:100A500057F005C056F004C055F003C054F02CD038
:100A6000060E3A5C29E127BC06D08B9A5B685A686F
:100A70005968586821D0827A949A02EE5CF0D89036
:100A80002D34E926000EEA22EECF07F0EFCF08F072
:100A900007503024036E08503120046E000E3220BF
:100AA000056E000E3320066E06C05BF005C05AF0DE
:100AB00004C059F003C058F017D833AE0BD0336AD6
:100AC000326A316A306A276A00EE40F01C0EEE6826
:100AD000E82EFDD706D033AE04D0336A326A316ACD
:100AE000306A817048EF01F03A68398E176A070E54
:100AF000175C33E2D8901734E96EEA6AEA36E936D1
:100B0000EA36400EE926000EEA22EFCF03F0ECCFE2
:100B100004F0ECCF05F0ECCF06F03650035C375014
:100B20000458385005583950065815E2D8901734F3
:100B3000E96EEA6AEA36E936EA36400EE926000E40
:100B4000EA22EFCF36F0ECCF37F0ECCF38F0ECCF35
:100B500039F017C03AF0172ACAE31200600E1D5C84
:100B600003E11EC029F027D0610E1D5C03E11EC009
:100B70002AF021D0620E1D5C03E0630E1D5C0AE1C9
:100B8000AF0E0DEC00F01D500DEC00F01E500DEC02
:100B900000F011D0780E1D5C03E11EC02BF00BD0CD
:100BA0007B0E1D5C03E11EC02CF005D07C0E1D5C8D
:100BB00002E11EC02DF01D6812002168120023689A
:100BC000120022681200070E1F5C0AE1BF0E0DEC36
:100BD00000F0070E0DEC00F020500DEC00F093D06B
:100BE000180E1F5C0AE1BF0E0DEC00F0180E0DECA4
:100BF00000F020500DEC00F086D0190E1F5C0AE1C9
:100C0000BF0E0DEC00F0190E0DEC00F020500DECB5
:100C100000F079D01E0E1F5C0DE120C029F020C02D
:100C20002AF020C02BF020C02CF020C02DF020C0D6
:100C30002EF069D0300E1F5C0AE1BF0E0DEC00F003
:100C4000300E0DEC00F020500DEC00F05CD0420EA8
:100C50001F5C13E1BF0E0DEC00F0420E0DEC00F036
:100C600020500DEC00F0205203E126904ED804D025
:100C7000929889888A84268046D0430E1F5C0AE1B8
:100C8000BF0E0DEC00F0430E0DEC00F020500DEC0B
:100C900000F039D0440E1F5C0AE1BF0E0DEC00F0ED
:100CA000440E0DEC00F020500DEC00F02CD0780E2E
:100CB0001F5C0DE1205020242F6E2FC002F0520E39
:100CC0000C6E080E0B6E010E11EC00F01CD07B0EAA
:100CD0001F5C19E1BF0E0DEC00F07B0E0DEC00F077
:100CE000000E0DEC00F0276A256A899A8B908B9292
:100CF000026A520E0C6E080E0B6E010E11EC00F023
:100D00008B968B988B9A1F681200929889988A9478
:100D1000256A276A296A2A6A2B6A2C6A2D6A2E6A32
:100D2000899A8B908B92026A520E0C6E080E0B6E93
:100D3000010E11EC00F07F0E2F6E8B968B988B9A24
:100D4000266A120002015D695C695C0E5F6F7A0EB3
:100D50005E6F590E616F850E606F580E636F140ED3
:100D6000626F560E656FA90E646F550E676F430E66
:100D7000666F530E696FE30E686F520E6B6F890ECC
:100D80006A6F510E6D6F350E6C6F4F0E6F6FE60E02
:100D90006E6F4E0E716F9C0E706F4D0E736F580E0E
:100DA000726F4C0E756F190E746F4A0E776FDF0EEF
:100DB000766F490E796FAA0E786F480E7B6F7A0EA8
:100DC0007A6F470E7D6F4F0E7C6F460E7F6F290E38
:100DD0007E6F450E816F080E806F430E836FEB0EA2
:100DE000826F420E856FD30E846F410E876FBF0EE8
:100DF000866F400E896FB00E886F3F0E8B6FA50E09
:100E00008A6F3E0E8D6F9E0E8C6F3D0E8F6F9C0E07
:100E10008E6F3C0E916F9E0E906F3B0E936FA40EE3
:100E2000926F3A0E956FAE0E946F390E976FBC0E9F
:100E3000966F380E996FCE0E986F370E9B6FE30E3C
:100E40009A6F360E9D6FFD0E9C6F360E9F6F1A0EB9
:100E50009E6F350EA16F3B0EA06F340EA36F5F0E19
:100E6000A26F330EA56F870EA46F320EA76FB20E5E
:100E7000A66F310EA96FE10EA86F310EAB6F140E85
:100E8000AA6F300EAD6F490EAC6F2F0EAF6F820E92
:100E9000AE6F2E0EB16FBE0EB06F2D0EB36FFD0E86
:100EA000B26F2D0EB56F3F0EB46F2C0EB76F850E5F
:100EB000B66F2B0EB96FCD0EB86F2B0EBB6F180E21
:100EC000BA6F2A0EBD6F670EBC6F290EBF6FB80ECA
:100ED000BE6F290EC16F0C0EC06F280EC36F620E5D
:100EE000C26F270EC56FBC0EC46F270EC76F180EDA
:100EF000C66F260EC96F760EC86F250ECB6FD80E43
:100F0000CA6F250ECD6F3C0ECC6F240ECF6FA20E94
:100F1000CE6F240ED16F0B0ED06F230ED36F760ED3
:100F2000D26F220ED56FE40ED46F220ED76F540EFF
:100F3000D66F210ED96FC60ED86F210EDB6F3B0E18
:100F4000DA6F200EDD6FB20EDC6F200EDF6F2B0E1E
:100F5000DE6F1F0EE16FA60EE06F1F0EE36F240E13
:100F6000E26F1E0EE56FA30EE46F1E0EE76F250EF7
:100F7000E66F1D0EE96FA90EE86F1D0EEB6F2E0ECA
:100F8000EA6F1C0EED6FB60EEC6F1C0EEF6F3F0E8E
:100F9000EE6F1B0EF16FCB0EF06F1B0EF36F580E42
:100FA000F26F1A0EF56FE80EF46F1A0EF76F790EE6
:100FB000F66F1A0EF96F0B0EF86F190EFB6FA00E7D
:100FC000FA6F190EFD6F360EFC6F180EFF6FCE0E06
:100FD000FE6F180E0301016F680E006F180E036F8D
:100FE000030E026F170E056FA00E046F170E076F2A
:100FF0003F0E066F160E096FDF0E086F160E0B6F91
:10100000800E0A6F160E0D6F240E0C6F150E0F6FEB
:10101000C80E0E6F150E116F6E0E106F150E136F3A
:10102000160E126F140E156FBF0E146F140E176F7D
:10103000690E166F140E196F150E186F130E1B6FB5
:10104000C20E1A6F130E1D6F710E1C6F130E1F6FE1
:10105000210E1E6F120E216FD20E206F120E236F03
:10106000840E226F120E256F380E246F110E276F1B
:10107000ED0E266F110E296FA30E286F110E2B6F28
:101080005A0E2A6F110E2D6F120E2C6F100E2F6F2D
:10109000CC0E2E6F100E316F870E306F100E336F27
:1010A000420E326F0F0E356F3469376FBD0E366FDB
:1010B0000F0E396F7C0E386F0F0E3B6F3D0E3A6F7F
:1010C0000E0E3D6FFE0E3C6F0E0E3F6FC00E3E6F5C
:1010D0000E0E416F830E406F0E0E436F470E426F30
:1010E0000E0E456F0C0E446F0D0E476FD20E466FFD
:1010F0000D0E496F990E486F0D0E4B6F610E4A6FC2
:101100000D0E4D6F2A0E4C6F0C0E4F6FF40E4E6F7E
:101110000C0E516FBE0E506F0C0E536F8A0E526F35
:101120000C0E556F560E546F0C0E576F230E566FE4
:101130000B0E596FF10E586F0B0E5B6FC00E5A6F8E
:101140005D695C69A20E5F6FC30E5E6F9A0E616F80
:10115000460E606F960E636F320E626F920E656F71
:101160003A0E646F8E0E676F5D0E666F8A0E696F42
:101170009A0E686F860E6B6FF00E6A6F830E6D6F3E
:101180005F0E6C6F7F0E6F6FE70E6E6F7C0E716F70
:10119000850E706F790E736F3B0E726F760E756FE2
:1011A000070E746F720E776FE80E766F6F0E796FA1
:1011B000DF0E786F6C0E7B6FEA0E7A6F6A0E7D6FB2
:1011C0000A0E7C6F670E7F6F3C0E7E6F640E816F20
:1011D000820E806F610E836FDA0E826F5F0E856FF5
:1011E000440E846F5C0E876FBF0E866F5A0E896F38
:1011F0004C0E886F570E8B6FE90E8A6F550E8D6FF0
:10120000960E8C6F530E8F6F8E6F510E916F200E56
:10121000906F4E0E936FFB0E926F4C0E956FE50E16
:10122000946F4A0E976FDC0E966F480E996FE20E20
:10123000986F460E9B6FF50E9A6F450E9D6F150EBB
:101240009C6F430E9F6F420E9E6F410EA16F7B0EEF
:10125000A06F3F0EA36FC00EA26F3E0EA56F100EC3
:10126000A46F3C0EA76F6D0EA66F3A0EA96FD40E39
:10127000A86F390EAB6F460EAA6F370EAD6FC20E58
:10128000AC6F360EAF6F490EAE6F340EB16FDA0E23
:10129000B06F330EB36F740EB26F320EB56F180E9F
:1012A000B46F300EB76FC50EB66F2F0EB96F7B0ED1
:1012B000B86F2E0EBB6F3A0EBA6F2D0EBD6F020EB9
:1012C000BC6F2B0EBF6FD10EBE6F2A0EC16FA90E61
:1012D000C06F290EC36F880EC26F280EC56F6F0EC8
:1012E000C46F270EC76F5E0EC66F260EC96F530EF2
:1012F000C86F250ECB6F500ECA6F240ECD6F540EE3
:10130000CC6F230ECF6F5E0ECE6F220ED16F6F0E9D
:10131000D06F210ED36F860ED26F200ED56FA30E25
:10132000D46F1F0ED76FC60ED66F1E0ED96FEF0E7D
:10133000D86F1E0EDB6FDA6F1D0EDD6F520EDC6F85
:101340001C0EDF6F8C0EDE6F1B0EE16FCB0EE06F9D
:101350001B0EE36F0F0EE26F1A0EE56F580EE46F6F
:10136000190EE76FA50EE66F180EE96FF80EE86F1D
:10137000180EEB6F4F0EEA6F170EED6FAB0EEC6FA2
:10138000170EEF6F0A0EEE6F160EF16F6F0EF06F05
:10139000150EF36FD70EF26F150EF56F430EF46F47
:1013A000140EF76FB30EF66F140EF96F270EF86F69
:1013B000130EFB6F9F0EFA6F130EFD6F1A0EFC6F6C
:1013C000120EFF6F990EFE6F120E0401016F1B0EBD
:1013D000006F110E036FA10E026F110E056F290E23
:1013E000046F100E076FB50E066F100E096F440ED6
:1013F000086F0F0E0B6FD60E0A6F0F0E0D6F6B0E70
:101400000C6F0F0E0F6F030E0E6F0E0E116F9D0EF1
:10141000106F0E0E136F3A0E126F0D0E156FDA0E5F
:10142000146F0D0E176F7C0E166F0D0E196F210EB7
:10143000186F0C0E1B6FC80E1A6F0C0E1D6F720EFC
:101440001C6F0C0E1F6F1E0E1E6F0B0E216FCC0E2D
:10145000206F0B0E236F7C0E226F0B0E256F2E0E4E
:10146000246F0A0E276FE30E266F0A0E296F990E5E
:10147000286F0A0E2B6F510E2A6F0A0E2D6F0B0E5E
:101480002C6F090E2F6FC80E2E6F090E316F850E4F
:10149000306F090E336F450E326F090E356F060E31
:1014A000346F080E376FC90E366F080E396F8E0E07
:1014B000386F080E3B6F540E3A6F080E3D6F1C0ECE
:1014C0003C6F070E3F6FE50E3E6F070E416FAF0E8C
:1014D000406F070E436F7B0E426F070E456F490E3C
:1014E000446F070E476F170E466F060E496FE70EE3
:1014F000486F060E4B6FB90E4A6F060E4D6F8B0E7E
:101500004C6F060E4F6F5F0E4E6F060E516F340E0E
:10151000506F060E536F0A0E526F050E556FE10E97
:10152000546F050E576FB90E566F050E596F930E17
:10153000586F050E5B6F6D0E5A6F00011200040E9E
:1015400001015F6F880E5E6F040E616FA60E606F03
:10155000040E636FB60E626F040E656FC60E646F85
:10156000040E676FD60E666F040E696FE60E686F25
:10157000040E6B6FF60E6A6F050E6D6F070E6C6FC3
:10158000050E6F6F170E6E6F050E716F280E706F60
:10159000050E736F390E726F050E756F4B0E746FFB
:1015A000050E776F5D0E766F050E796F6E0E786F94
:1015B000050E7B6F800E7A6F050E7D6F930E7C6F2C
:1015C000050E7F6FA50E7E6F050E816FB80E806FC2
:1015D000050E836FCB0E826F050E856FDF0E846F55
:1015E000050E876FF20E866F060E896F886F8B6F00
:1015F0001A0E8A6F060E8D6F2E0E8C6F060E8F6F71
:10160000430E8E6F060E916F580E906F060E936FFD
:101610006D0E926F060E956F830E946F060E976F88
:10162000980E966F060E996FAE0E986F060E9B6F12
:10163000C40E9A6F060E9D6FDB0E9C6F060E9F6F99
:10164000F20E9E6F070EA16F090EA06F070EA36F1B
:10165000210EA26F070EA56F380EA46F070EA76F9D
:10166000500EA66F070EA96F690EA86F070EAB6F1D
:10167000810EAA6F070EAD6F9A0EAC6F070EAF6F9B
:10168000B40EAE6F070EB16FCD0EB06F070EB36F15
:10169000E70EB26F080EB56F020EB46F080EB76F8B
:1016A0001D0EB66F080EB96F380EB86F080EBB6FFF
:1016B000530EBA6F080EBD6F6F0EBC6F080EBF6F72
:1016C0008B0EBE6F080EC16FA70EC06F080EC36FE2
:1016D000C40EC26F080EC56FE10EC46F080EC76F4F
:1016E000C669090EC96F1D0EC86F090ECB6F3B0E80
:1016F000CA6F090ECD6F5A0ECC6F090ECF6F790EDF
:10170000CE6F090ED16F990ED06F090ED36FB90E3F
:10171000D26F090ED56FD90ED46F090ED76FFA0E9E
:10172000D66F0A0ED96F1B0ED86F0A0EDB6F3D0EF7
:10173000DA6F0A0EDD6F5F0EDC6F0A0EDF6F820E4E
:10174000DE6F0A0EE16FA50EE06F0A0EE36FC80EA2
:10175000E26F0A0EE56FEC0EE46F0B0EE76F110EF1
:10176000E66F0B0EE96F360EE86F0B0EEB6F5B0E3C
:10177000EA6F0B0EED6F810EEC6F0B0EEF6FA70E85
:10178000EE6F0B0EF16FCE0EF06F0B0EF36FF50ECA
:10179000F26F0C0EF56F1D0EF46F0C0EF76F460E08
:1017A000F66F0C0EF96F6F0EF86F0C0EFB6F980E44
:1017B000FA6F0C0EFD6FC20EFC6F0C0EFF6FED0E7C
:1017C000FE6F0D0E0201016F180E006F0D0E036FFC
:1017D000430E026F0D0E056F700E046F0D0E076F36
:1017E0009C0E066F0D0E096FCA0E086F0D0E0B6F63
:1017F000F80E0A6F0E0E0D6F260E0C6F0E0E0F6F89
:10180000550E0E6F0E0E116F850E106F0E0E136FAC
:10181000B60E126F0E0E156FE70E146F0F0E176FC8
:10182000180E166F0F0E196F4B0E186F0F0E1B6FE1
:101830007E0E1A6F0F0E1D6FB10E1C6F0F0E1F6FF5
:10184000E60E1E6F100E216F1B0E206F100E236F01
:10185000500E226F100E256F870E246F100E276F0B
:10186000BE0E266F100E296FF60E286F110E2B6F0D
:101870002E0E2A6F110E2D6F680E2C6F110E2F6F0A
:10188000A20E2E6F110E316FDC0E306F120E336F01
:10189000180E326F120E356F540E346F120E376FF2
:1018A000910E366F120E396FCF0E386F130E3B6FDD
:1018B0000E0E3A6F130E3D6F4D0E3C6F130E3F6FC1
:1018C0008E0E3E6F130E416FCF0E406F140E436F9E
:1018D000110E426F140E456F540E446F140E476F75
:1018E000980E466F140E496FDC0E486F150E4B6F45
:1018F000220E4A6F150E4D6F680E4C6F150E4F6F0E
:10190000B00E4E6F150E516FF80E506F160E536FCE
:10191000410E526F160E556F8C0E546F160E576F88
:10192000D70E566F170E596F230E586F170E5B6F39
:0A193000700E5A6F00011200FFD77D
:020000040030CA
:0300010006160ED2
:020005008580F4
:060008000FC00FE00F40E5
:00000001FF
